BL51 BANKED LINKER/LOCATER V6.22                                                        08/21/2014  16:46:16  PAGE 1


BL51 BANKED LINKER/LOCATER V6.22, INVOKED BY:
C:\KEIL\C51\BIN\BL51.EXE inter2.obj TO inter2


INPUT MODULES INCLUDED:
  inter2.obj (INTER2)


LINK MAP OF MODULE:  inter2 (INTER2)


            TYPE    BASE      LENGTH    RELOCATION   SEGMENT NAME
            -----------------------------------------------------

            * * * * * * *   D A T A   M E M O R Y   * * * * * * *
            REG     0000H     0008H     ABSOLUTE     "REG BANK 0"

            * * * * * * *   C O D E   M E M O R Y   * * * * * * *
            CODE    0000H     008DH     ABSOLUTE     



SYMBOL TABLE OF MODULE:  inter2 (INTER2)

  VALUE           TYPE          NAME
  ----------------------------------

  -------         MODULE        INTER2
  D:00E0H         SYMBOL        ACC
  C:007EH         SYMBOL        DEALY
  B:00A8H.7       SYMBOL        EA
  B:00A8H.0       SYMBOL        EX0
  B:00A8H.2       SYMBOL        EX1
  C:0054H         SYMBOL        FLASH
  C:006DH         SYMBOL        FLASH1
  C:004CH         SYMBOL        INTER0
  C:0065H         SYMBOL        INTER1
  D:00B8H         SYMBOL        IP
  B:0088H.0       SYMBOL        IT0
  B:0088H.2       SYMBOL        IT1
  C:003DH         SYMBOL        LOOP
  C:0080H         SYMBOL        LOOP1
  C:0082H         SYMBOL        LOOP2
  C:0084H         SYMBOL        LOOP3
  C:0030H         SYMBOL        MAIN
  D:0090H         SYMBOL        P1
  C:0000H         LINE#         2
  C:0003H         LINE#         4
  C:0013H         LINE#         6
  C:0030H         LINE#         8
  C:0032H         LINE#         9
  C:0034H         LINE#         10
  C:0036H         LINE#         11
  C:0038H         LINE#         12
  C:003AH         LINE#         13
  C:003DH         LINE#         14
  C:0040H         LINE#         15
  C:0043H         LINE#         16
BL51 BANKED LINKER/LOCATER V6.22                                                      08/21/2014  16:46:16  PAGE 2


  C:0046H         LINE#         17
  C:0049H         LINE#         18
  C:004CH         LINE#         20
  C:004EH         LINE#         21
  C:0050H         LINE#         22
  C:0052H         LINE#         23
  C:0054H         LINE#         24
  C:0056H         LINE#         25
  C:0059H         LINE#         26
  C:005BH         LINE#         27
  C:005CH         LINE#         28
  C:005FH         LINE#         29
  C:0062H         LINE#         30
  C:0064H         LINE#         31
  C:0065H         LINE#         33
  C:0067H         LINE#         34
  C:0069H         LINE#         35
  C:006BH         LINE#         36
  C:006DH         LINE#         37
  C:006FH         LINE#         38
  C:0072H         LINE#         39
  C:0074H         LINE#         40
  C:0075H         LINE#         41
  C:0078H         LINE#         42
  C:007BH         LINE#         43
  C:007DH         LINE#         44
  C:007EH         LINE#         45
  C:0080H         LINE#         46
  C:0082H         LINE#         47
  C:0084H         LINE#         48
  C:0085H         LINE#         49
  C:0086H         LINE#         50
  C:0088H         LINE#         51
  C:008AH         LINE#         52
  C:008CH         LINE#         53
  -------         ENDMOD        INTER2

Program Size: data=8.0 xdata=0 code=141
LINK/LOCATE RUN COMPLETE.  0 WARNING(S),  0 ERROR(S)
